:020000002928AD
:08000800FF00030E8301A000BC
:100010000A08A1008A010408A2000E28B8080319E2
:10002000B703B80B1F28B708031D1F280F30B700F0
:100030004230B8004030B9070318B80AAC240B119D
:100040002208840021088A00200E8300FF0E7F0E04
:100050000900FF30A500FF30A600FF30A700FF30E9
:10006000A8000F30A9008A110A12C7270A308A1186
:100070000A12E8272A128A150A124B2003308A1125
:100080000A12B62732308A150A12142003308A1158
:100090000A12B62732308A150A12142003308A1148
:1000A0000A12B62732308A150A12142032308A1109
:1000B0000A12A02728308A110A12A0278A110A12D0
:1000C0005A278A110A120A278A110A125627271359
:1000D0008A150A126D20A7178A150A126A208A1536
:1000E0000A12962024309800193099008A150A12B5
:1000F0009920903098001A081A081A0800309900C0
:10010000AD01AE010F30B7004230B8004030B90049
:10011000A7128A150A12702026138A150A127C204B
:10012000A6138A150A127920AA138A150A124220E8
:100130002A138A150A124520AB168A150A1239208D
:1001400001308A110A12DF27AB128A150A123920F0
:100150008A150A1237208A150A12962088308A15C5
:100160000A1292208A150A12992081018B178B1688
:100170008A110A120E25FF308A150A1285208A116B
:100180000A120719ED2A01308A110A12DF278A1193
:100190000A120719ED2AAB168A150A123920013006
:1001A0008A110A12DF27AB128A150A1239208A1126
:1001B0000A1272278A110A120719E1288A110A12F3
:1001C000DA2801308A110A12DF27B601B5018A1137
:1001D0000A120719EE288A110A12C62A3A08013CA7
:1001E0008A110A12031DC32ABA011F3036028A116E
:1001F0000A12031C0229AA178A150A1242208A1120
:100200000A120629AA138A150A124220B401FF30E5
:100210008A110A121D26FF30B40700308A110A1213
:10022000DC258A110A126E2741308A110A129227A0
:100230002D08BE002E088A110A12D8243B08B100EE
:100240003C08B2003D08B30032088A110A121D268C
:100250003208B40733088A110A121D263308B4077E
:100260001F3036028A110A1203185829AE30BB001B
:100270003608BC003508BD0032088A110A1228264B
:1002800001308A110A12E8278A110A129F24AE301F
:10029000BB003608BC003508BD0033088A110A12BD
:1002A000282601308A110A12E8278A110A129F248F
:1002B0003208BB0033088A110A12AF2401308A11B8
:1002C0000A12DC2542308A110A1292272D08BE003C
:1002D0002E088A110A12D8243B08B1003C08B2004B
:1002E0003D08B30032088A110A121D263208B407ED
:1002F00033088A110A121D263308B4071F3036024C
:100300008A110A120318A629AE30BB003608BC00B9
:100310003508BD0032088A110A12282601308A11D8
:100320000A12E8278A110A129F24AE30BB00360851
:10033000BC003508BD0033088A110A122826013096
:100340008A110A12E8278A110A129F243208BB0078
:1003500033088A110A12AF2402308A110A12DC25EE
:1003600043308A110A1292272D08BE002E088A11E6
:100370000A12D8243B08B1003C08B2003D08B30083
:1003800032088A110A121D263208B40733088A116E
:100390000A121D263308B4071F3036028A110A12CA
:1003A0000318F429AE30BB003608BC003508BD0088
:1003B00032088A110A12282601308A110A12E82707
:1003C0008A110A129F24AE30BB003608BC003508E3
:1003D000BD0033088A110A12282601308A110A1238
:1003E000E8278A110A129F243208BB0033088A11B9
:1003F0000A12AF248A110A126A2703308A110A12DC
:10040000DC2544308A110A1292272D08BE002E08DE
:100410008A110A12D8243B08B1003C08B2003D08FA
:10042000B30032088A110A121D263208B4073308B5
:100430008A110A121D263308B4071F3036028A11AA
:100440000A120318452AAE30BB003608BC00350836
:10045000BD0032088A110A12282601308A110A12B8
:10046000E8278A110A129F24AE30BB003608BC0070
:100470003508BD0033088A110A12282601308A1176
:100480000A12E8278A110A129F243208BB00330897
:100490008A110A12AF2404308A110A12DC25453071
:1004A0008A110A1292272D08BE002E088A110A12FC
:1004B000D8243B08B1003C08B2003D08B300320824
:1004C0008A110A121D263208B40733088A110A124B
:1004D0001D263308B4071F3036028A110A1203188A
:1004E000932AAE30BB003608BC003508BD00320888
:1004F0008A110A12282601308A110A12E8278A1165
:100500000A129F24AE30BB003608BC003508BD007F
:1005100033088A110A12282601308A110A12E827A4
:100520008A110A129F243208BB0033088A110A126A
:10053000AF2420308A110A12922752308A110A12EF
:10054000922745308A110A12922743308A110A12E3
:1005500092273408F039B00030088A110A121D269B
:1005600034080F39B00030088A110A121D262A17E4
:100570008A150A12452001308A110A12DF272A1330
:100580008A150A1245208A110A12E728AB168A1525
:100590000A12392001308A110A12DF27AB128A159C
:1005A0000A123920AE30BB003608BC003508BD0049
:1005B000FF308A110A12282601308A110A12E82710
:1005C0008A110A1272278A110A120E258A110A123A
:1005D0000719ED2A8A110A12E62A8A110A128718C7
:1005E000992C01308A110A12DF278A110A12871802
:1005F000992CAB168A150A12392001308A110A1279
:10060000DF27AB128A150A1239208A110A127227C3
:100610008A110A1287180F2B8A110A12082B01302F
:100620008A110A12DF278A110A1272272A178A15DD
:100630000A124520B601B5011F3036028A110A128E
:100640000318262B8A110A128718292B8A110A12DD
:100650007C2CB401FF308A110A121D26FF30B4072A
:10066000AE30BB003608BC003508BD008A110A1246
:1006700045263E08AC002C08B2008A110A129F24BD
:10068000AE30BB003608BC003508BD008A110A1226
:1006900045263E08AC002C08B3008A110A129F249C
:1006A0008A110A126E2741308A110A1292273208E3
:1006B0008A110A121D263208B40733088A110A1259
:1006C0001D263308B4073208BB0033088A110A120A
:1006D000AF24AE30BB003608BC003508BD008A111F
:1006E0000A1245263E08AC002C08B2008A110A12F4
:1006F0009F24AE30BB003608BC003508BD008A110F
:100700000A1245263E08AC002C08B3008A110A12D2
:100710009F2442308A110A12922732088A110A1243
:100720001D263208B40733088A110A121D26330821
:10073000B4073208BB0033088A110A12AF24AE3066
:10074000BB003608BC003508BD008A110A124526D8
:100750003E08AC002C08B2008A110A129F24AE3069
:10076000BB003608BC003508BD008A110A124526B8
:100770003E08AC002C08B3008A110A129F244330B3
:100780008A110A12922732088A110A121D2632088B
:10079000B40733088A110A121D263308B407320839
:1007A000BB0033088A110A12AF248A110A126A2781
:1007B000AE30BB003608BC003508BD008A110A12F5
:1007C00045263E08AC002C08B2008A110A129F246C
:1007D000AE30BB003608BC003508BD008A110A12D5
:1007E00045263E08AC002C08B3008A110A129F244B
:1007F00044308A110A12922732088A110A121D26E1
:100800003208B40733088A110A121D263308B407C8
:100810003208BB0033088A110A12AF24AE30BB0085
:100820003608BC003508BD008A110A1245263E086C
:10083000AC002C08B2008A110A129F24AE30BB0013
:100840003608BC003508BD008A110A1245263E084C
:10085000AC002C08B3008A110A129F24AE30BB00F2
:100860003608BC003508BD008A110A1245263E082C
:10087000AC002C08FF3C8A110A12031D412C1F30CA
:10088000B60045308A110A12922732088A110A12DC
:100890001D263208B40733088A110A121D263308B0
:1008A000B4073208BB0033088A110A12AF24203083
:1008B0008A110A12922750308A110A1292274C305C
:1008C0008A110A12922741308A110A12922759304E
:1008D0008A110A1292273408F039B00030088A11C0
:1008E0000A121D2634080F39B00030088A110A1286
:1008F0001D268A110A121C2BAB168A150A123920E2
:1009000001308A110A12DF27AB128A150A12392028
:100910008A110A1272278A110A120E252A138A15C1
:100920000A1245208A110A128718992C8A110A1274
:10093000922C8A110A12BF288A110A129C2C35089F
:10094000FF3C8A110A12031DAA2CB501B60A8A11AE
:100950000A12AB2CB50A08000130BA000800BC002E
:100960003B08AF002F0E0F39AF003030AF072F0814
:100970008A110A1292273B080F39AF003030AF07B7
:100980002F088A110A1292273C08AF002F0E0F3948
:10099000AF003030AF072F088A110A1292273C08A7
:1009A0000F39AF003030AF072F088A110A12922F8B
:1009B000BF00BB01BC01BD011030C0003D088A1161
:1009C0000A12FA244108BD003C088A110A12FA24CE
:1009D0004108BC003B088A110A12FA244108BB00F6
:1009E000BF0DBE0DBD0DBC0DBB0D8A110A12C00B93
:1009F000DE2C0800C1004108033EC2008A110A1221
:100A0000C21D042D4208C1004108303EC2008A11B7
:100A10000A12C21F0D2D4208C10008008A110A12D5
:100A2000722720308A110A12922720308A110A1266
:100A3000922720308A110A12922754308A110A1202
:100A4000922765308A110A1292276C308A110A1295
:100A5000922765308A110A1292276D308A110A1284
:100A6000922765308A110A12922774308A110A126D
:100A7000922772308A110A12922769308A110A125B
:100A8000922763308A110A1292278A110A126A2762
:100A900020308A110A12922720308A110A129227D6
:100AA00053308A110A12922779308A110A1292273A
:100AB00073308A110A12922774308A110A1292270F
:100AC00065308A110A1292276D308A110A12922714
:100AD00020308A110A12922772308A110A12922744
:100AE00065308A110A12922761308A110A12922700
:100AF00064308A110A12922779308A110A129227D9
:100B000054308A110A121D2665308A110A121D26D8
:100B10006C308A110A121D2665308A110A121D26B0
:100B20006D308A110A121D2665308A110A121D269F
:100B300074308A110A121D2672308A110A121D267B
:100B400069308A110A121D2663308A110A121D2685
:100B500020308A110A121D2653308A110A121D26CE
:100B600079308A110A121D2673308A110A121D2645
:100B700074308A110A121D2665308A110A121D2648
:100B80006D308A110A121D2620308A110A121D2684
:100B900072308A110A121D2665308A110A121D262A
:100BA00061308A110A121D2664308A110A121D262C
:100BB00079308A110A121D2EBB00BB088A110A1255
:100BC000031DE42D4130BB003B08013C8A110A1291
:100BD000031DEC2D4930BB003B08023C8A110A1270
:100BE000031DF42D5130BB003B08033C8A110A124F
:100BF000031DFC2D5930BB003B08043C8A110A122E
:100C0000031D042E6130BB003B089F0001308A1198
:100C10000A12F1278316031382309F0083123B08C8
:100C20009F001F151F19122E1E08AD0083160313F7
:100C30001E088312AE0083120800BB003B080C1E86
:100C40001F2E8B138B1B212E99008B170800080079
:100C5000BE003B088A110A1264263C088A110A1257
:100C600097268A110A12AA263D088A110A12972687
:100C70008A110A12AA263E088A110A1297268A1198
:100C80000A12AA268A110A120A2FBE003B088A11EC
:100C90000A1264263C088A110A1297268A110A123F
:100CA000AA263D088A110A1297268A110A12AA2634
:100CB0003B088A110A126F268A110A127B263F0806
:100CC000BE008A110A120A2FBF008A110A123027A9
:100CD0003F088A110A1297268A110A12AA2EBF000B
:100CE0008A110A1230273F08013E8A110A129726FC
:100CF0008A110A12AA2EBF008A110A12CC263F10AE
:100D00008A110A12A31C852E3F140830C00003105C
:100D1000BF0D8A110A12CC263F108A110A12A31C99
:100D2000922E3F148A110A12C00B872E0800C000B1
:100D30000830C100A3108A110A12C01FA02EA314EC
:100D40008A110A12ED260310C00D8A110A12C10B76
:100D50009A2E08008A110A12562727168A150A1297
:100D600073208A110A125627A7158A150A127620AF
:100D70008A110A1256278A110A128719C22E8A115D
:100D80000A12BB2E8A110A125627A7118A150A12B7
:100D900076208A110A12562F8A110A125627271610
:100DA0008A150A1273208A110A125627A3108A1173
:100DB0000A12071EDC2EA3148A110A125627A71145
:100DC0008A150A1276208A110A125627A7158A1543
:100DD0000A1276208A110A12562F8A110A125627F1
:100DE00027128A110A12A31CF62E27168A150A1238
:100DF00073208A110A125627A7158A150A1276201F
:100E00008A110A125627A7118A150A1276208A110A
:100E10000A12562F8A110A125627A7118A150A128A
:100E200076208A110A12562727128A150A12732071
:100E30008A110A125627A7158A150A1276208A11D6
:100E40000A12562727168A150A1273208A110A12C7
:100E50005627A7118A150A1276208A110A12562FD0
:100E60008A110A125627A7118A150A1276208A11AA
:100E70000A12562727168A150A1273208A110A1297
:100E80005627A7158A150A1276208A110A125627A4
:100E900027128A150A1273208A110A125627A711DF
:100EA0008A150A1276208A110A12562F0C308A15DA
:100EB0000A122828AB118A150A123F20A7118A1599
:100EC0000A1276202B128A150A123C2027128A1544
:100ED0000A127328A8308A110A12A02F80308A11B2
:100EE0000A12A02F08308A110A12A02701308A1195
:100EF0000A12A027C8308A150A12142002308A115B
:100F00000A12A027C8308A150A12142006308A1146
:100F10000A12A0270C308A110A12A027C8308A159D
:100F20000A121428BD002A168A150A124B203D0EFB
:100F30000F398A110A12B6273D088A110A12B62FF4
:100F4000BB002A128A150A124B203B0E0F398A1158
:100F50000A12B62782308A150A1214203B088A1119
:100F60000A12B62782308A150A121428BE00AA1661
:100F70008A150A1248203E088A150A124E20AA1223
:100F80008A150A124820FA308A150A1228280030D9
:100F90008A150A124E202A128A150A124B20AA120A
:100FA0008A150A12482000308A150A125F2026127C
:100FB0008A150A128220A6128A150A127F28BB00FF
:100FC0003B08BD006430BE000A308A110A12FA2FB5
:100FD000BB003B08BD006430BE0001308A110A121C
:100FE000FA2FBC003C08BD000A30BE0001308A1157
:100FF0000A12FA2FBF00FF30C0003E08C2003D08B1
:10100000C10017308A150A124007031804288A15F0
:101010000A12C10B01288A110A12C20BFF2F8A1172
:101020000A12BF0BFD2F0800BC003C08BD00BD0824
:101030008A150A12031D1F288A150A1227280A304A
:101040008A150A122820BD038A150A1217280800DB
:10105000C200F430C300FC30C4008A150A124208F2
:101060004307031C003444070318332808006400B6
:1010700008008A150A1259288A150A1259288A1551
:101080000A1259288A150A125C288A150A125C2845
:101090008A150A125C288A150A125C28BF003F08CC
:1010A0000F39C0002A08F0394004AA008A150A1234
:1010B0005C282B08870008002A0886000800AC007E
:1010C0002C080F39AD002608F0392D04A6008A152A
:1010D0000A128C288A150A1289288A150A12892868
:1010E0008A150A1289288A150A1289288A150A126D
:1010F00089288A150A128C288A150A128C288A15C2
:101100000A128C288A150A128C28A5008A150A1240
:101110008F282708670008002608660008002508B1
:1011200065000800BB003B0862000800831603133B
:081130000800831203130800FC
:02400E00723FFF
:00000001FF
